:100000000C9434000C944F000C944F000C944F004F
:100010000C944F000C944F000C944F000C944F0024
:100020000C944F000C944F000C944F000C944F0014
:100030000C944F000C944F000C944F000C944F0004
:100040000C944F000C944F000C947F000C944F00C4
:100050000C944F000C944F000C944F000C944F00E4
:100060000C944F000C944F0011241FBECFEFD4E02E
:10007000DEBFCDBF11E0A0E0B1E0E8E2F1E002C0F8
:1000800005900D92A030B107D9F711E0A0E0B1E0E2
:1000900001C01D92A130B107E1F70C9463000C94EC
:1000A0000000209A08959C01832F99278093C50012
:1000B0002093C4001092C00088E98093C1008EE0B4
:1000C0008093C2000895CFEFD4E0DEBFCDBF0E9481
:1000D000510083E390E00E9453007894289A809125
:1000E00000018823E1F38091C00085FFFCCF80915F
:1000F00000018093C600109200012898F0CF1F9253
:100100000F920FB60F9211248F93289A8091C000FE
:1001100084FD04C08091C600809300018F910F90F0
:080120000FBE0F901F9018950F
:00000001FF
